:020000040800F2
:1000000000500020CD0B00083D0100084101000810
:1000100045010008490100084D01000800000000EA
:100020000000000000000000000000005101000876
:100030005501000800000000590100085D0100089A
:10004000110C0008110C0008110C0008110C00081C
:10005000110C0008110C0008110C0008110C00080C
:10006000110C0008110C0008110C0008110C0008FC
:10007000110C0008110C0008110C0008110C0008EC
:10008000110C0008110C0008110C0008110C0008DC
:10009000110C0008110C0008110C0008110C0008CC
:1000A000110C0008110C0008110C0008110C0008BC
:1000B000110C0008110C0008110C0008110C0008AC
:1000C000110C0008110C0008110C0008110C00089C
:1000D000110C0008110C0008110C0008110C00088C
:1000E000110C0008110C0008110C000800000000A1
:1000F0000000000000000000000000000000000000
:0C01000000000000000000005FF808F1A3
:10010C0040F21403C2F200031A780AB901201870E5
:10011C00704700BF40F21400C2F2000008B503683B
:10012C002BB140F20003C0F2000303B1984708BDA5
:10013C00704700BFFEE700BFFEE700BFFEE700BF51
:10014C00FEE700BF704700BF704700BF704700BF9D
:10015C00704700BFCB7810B413F0100F18BF8A781B
:10016C0003F00F0C18BF4CEA020C0A8812F0FF0FB8
:10017C0029D002F001040168002C40F0258102F026
:10018C000204002C40F0FD8002F00404002C40F02E
:10019C00098102F00804002C40F0AE8002F010043B
:1001AC00002C40F0BA8002F02004002C40F0C680F5
:1001BC0002F04004002C40F0D28002F08004002CAD
:1001CC0040F014810160FF2A20D902F48074416848
:1001DC00002C27D102F40074002C32D102F480647C
:1001EC00002C3DD102F40064002C48D102F4805460
:1001FC00002C53D102F40054002C5ED102F4804444
:10020C00002C69D102F4004212B9416010BC704755
:10021C00282B6CF31F7108BF4261F6D0482B08BF26
:10022C000261F2E721F00F01282B4CEA010108BF13
:10023C004461CFD0482B08BF046102F40074002C39
:10024C00CCD021F0F001282B41EA0C1108BF4461FD
:10025C00C4D0482B08BF046102F48064002CC1D0C8
:10026C0021F47061282B41EA0C2108BF4461B9D0FC
:10027C00482B08BF046102F40064002CB6D021F4B2
:10028C007041282B41EA0C3108BF4461AED0482B99
:10029C0008BF046102F48054002CABD021F470210F
:1002AC00282B41EA0C4108BF4461A3D0482B08BF5E
:1002BC00046102F40054002CA0D021F47001282B0E
:1002CC0041EA0C5108BF446198D0482B08BF046127
:1002DC0002F48044002C95D021F07061282B41EA67
:1002EC000C6108BF44618DD0482B02F4004208BF5A
:1002FC000461002A89D08BE721F47041282B41EA54
:10030C000C3108BF44613FF449AF482B08BF04616E
:10031C0002F01004002C3FF446AF21F47021282B7E
:10032C0041EA0C4108BF44613FF43DAF482B08BF84
:10033C00046102F02004002C3FF43AAF21F4700168
:10034C00282B41EA0C5108BF44613FF431AF482BD4
:10035C0008BF046102F04004002C3FF42EAF21F0E2
:10036C007061282B41EA0C6108BF44613FF425AF52
:10037C00482B08BF046102F08004002C3FF422AF2C
:10038C0034E021F0F001282B41EA0C1108BF446144
:10039C003FF4FAAE482B08BF046102F00404002CB1
:1003AC003FF4F7AE21F47061282B41EA0C2108BF11
:1003BC0044613FF4EEAE482B08BF046102F0080420
:1003CC00002C3FF4EBAE97E721F00F01282B4CEA01
:1003DC00010108BF44613FF4D2AE482B08BF046151
:1003EC0002F00204002C3FF4CFAECAE7282B6CF3CA
:1003FC001F7108BF44613FF4E5AE482B08BF046190
:10040C00E0E600BF042202214FF0FF33C27081707E
:10041C0003807047836819420CBF0020012070478D
:10042C00806880B2704700BFC36819420CBF0020BF
:10043C0001207047C06880B2704700BF01617047EF
:10044C00416170470AB9416170470161704700BF53
:10045C00C160704741F4803383618161836183693A
:10046C008369704740F20002C4F2010210B44FF6E7
:10047C0080731468C0F2000304EA030C41EA001113
:10048C0041EA0C03136010BC704700BF40F21C0320
:10049C00C4F220231860704740F200030028C4F215
:1004AC000103B4BFDA695A6800F44013B3F5401F76
:1004BC0010B41FFA80FC25D010F4801F19D0C0F3A3
:1004CC000343032414FA03F322EA030242F070629A
:1004DC0029B1430D19010CFA01FC42EA0C02002867
:1004EC0040F20000C4F20100B4BFC261426010BC13
:1004FC007047430D1B010CFA03F322EA030242F08E
:10050C007062E5E740F20003C4F201035C6822F07C
:10051C00706224F070645C60DAE700BF01F00303E2
:10052C0010B40F229C00A24010FA04F3890840F288
:10053C000004C4F20104023154F8210020EA020242
:10054C0044F8212054F82120134344F8213010BCE6
:10055C00704700BF40F2DC03C4F2202318607047E0
:10056C000120014610B500F00BFA01200021BDE876
:10057C00104000F005BA00BF40F60003C4F20103BE
:10058C00984210B530D040F60041C4F201018842C7
:10059C0034D041F20002C4F20102904238D041F250
:1005AC00004CC4F2010C60453CD041F60003C4F28F
:1005BC000103984240D041F60041C4F20101884247
:1005CC0044D042F20002C4F20102904200D010BDAD
:1005DC0001214FF4807000F0D3F94FF480700021AA
:1005EC00BDE8104000F0CCB90420012100F0C8F99E
:1005FC0004200021BDE8104000F0C2B90820012100
:10060C0000F0BEF908200021BDE8104000F0B8B998
:10061C001020012100F0B4F910200021BDE8104099
:10062C0000F0AEB92020012100F0AAF92020002111
:10063C00BDE8104000F0A4B94020012100F0A0F961
:10064C0040200021BDE8104000F09AB98020012123
:10065C0000F096F980200021BDE8104000F090B920
:10066C0041F20003C4F20203186840F2000C40F09F
:10067C0001021A605968CFF6FF0C01EA0C005860B1
:10068C001A6822F0847C2CF480311960186820F4EC
:10069C0080221A6059684FF41F0221F4FE00586042
:1006AC009A60704741F20003C4F202031968B0F576
:1006BC00803F21F480321A60196821F480221A607C
:1006CC0007D0B0F5802F03D1186840F4A021196031
:1006DC0070471A6842F480301860704782B041F25B
:1006EC00000100230193C4F202010A680198431C23
:1006FC0001930198B0F5A06F02D012F4003FF4D032
:10070C0041F20002C4F202021168C1F3404002B08F
:10071C00704700BF41F20003C4F202031A6822F0D2
:10072C00F80141EAC0021A60704700BF40F20003B2
:10073C00C4F242231860704741F20003C4F2020372
:10074C005A6822F47C1C40EA0C020A435A60704737
:10075C0040F26003C4F242231860704741F2000378
:10076C00C4F202035A6822F0030140EA01025A6003
:10077C00704700BF41F20003C4F20203586800F056
:10078C000C00704741F20003C4F202035A6822F0D5
:10079C00F00140EA01025A60704700BF41F20003C9
:1007AC00C4F202035A6822F4E06140EA01025A6082
:1007BC00704700BF41F20003C4F202035A6822F4EE
:1007CC00605141EAC0025A60704700BF49B941F21A
:1007DC000901C4F2020191F800C02CEA0000087073
:1007EC00704741F20903C4F202031A7810431870DF
:1007FC00704700BF40F2D803C4F242231860704720
:10080C0041F20003C4F202035A6822F4404140EA68
:10081C0001025A60704700BF41F220030022C4F26B
:10082C00020301281A701A7004D0042801D1052083
:10083C00187070471870704740F28043C4F242231E
:10084C001860704741F20003C4F20203196A40EACF
:10085C0001021A62704700BF40F23C43C4F24223CB
:10086C001860704741F20003C4F202035A6810B4D6
:10087C0002F00C02042A01D0082A2ED041F20021E9
:10088C00C0F27A01016041F20002C4F20202546823
:10089C0040F20003C2F20003C4F3031C13F80CC0B3
:1008AC0021FA0CF141605468C4F3022C13F80C408B
:1008BC0031FA04F484605468C4F3C22C13F80CC0ED
:1008CC0021FA0CF1C1605268C2F38132D3181A7C40
:1008DC00B1FBF2F1016110BC70475A685C68C2F35D
:1008EC008341023114F4803F0BD05B6813F4003F5A
:1008FC0007D141F20024C0F27A0404FB01F101603B
:10090C00C1E740F6001CC0F23D0C0CFB01F101608C
:10091C00B9E700BF41B941F20001C4F202014B69D1
:10092C0023EA00004861704741F20003C4F202035D
:10093C005A6910435861704741B941F20001C4F241
:10094C0002018B6923EA00008861704741F20003C1
:10095C00C4F202039A6910439861704741B941F29D
:10096C000001C4F20201CB6923EA0000C8617047A0
:10097C0041F20003C4F20203DA691043D8617047F4
:10098C0041B941F20001C4F20201CB6823EA000034
:10099C00C860704741F20003C4F20203DA681043E6
:1009AC00D860704741B941F20001C4F202010B69F1
:1009BC0023EA00000861704741F20003C4F202030D
:1009CC001A6910431861704740F24043C4F2422345
:1009DC001860704740F24C03C4F242231860704711
:1009EC0041F20703C4F20203187070474309012B4C
:1009FC000ED0022B41F20003C4F202030CBF1B6A9F
:100A0C005B6A00F01F0133FA01F000F0010070473F
:100A1C0041F20003C4F202031B6800F01F0133FA19
:100A2C0001F000F00100704741F20003C4F2020330
:100A3C00586A40F080725A62704700BF41F2000160
:100A4C00C4F202018B6818420CBF002001207047D1
:100A5C0041F20A03C4F202031870704782B001908D
:100A6C00019B2BB1019A511E019101980028F9D1DB
:100A7C0002B0704710B5FFF7F3FD4FF48030FFF76D
:100A8C0011FEFFF72BFE40F21803C2F200030128FF
:100A9C000446187000D010BD0020FFF773FE002034
:100AAC00FFF788FE4FF48060FFF778FE4FF480303C
:100ABC000021FFF741FE2046FFF74AFE3920FFF7E1
:100ACC0095FF0028FAD00220FFF748FEFFF752FEF0
:100ADC000828FBD110BD00BF08B541F20000C4F2DC
:100AEC0001002021FFF7AAFC41F20000C4F2010032
:100AFC001021FFF7A5FC40F60040C4F20100802154
:100B0C00FFF79CFC40F60040C4F201004FF48071EA
:100B1C00FFF796FC4FF6FE73C0F21F03023BFDD1AC
:100B2C0041F20000C4F201001021FFF787FC41F2F2
:100B3C000000C4F201002021FFF782FC40F60040C7
:100B4C00C4F201004FF48071FFF778FC40F60040CE
:100B5C00C4F201008021FFF773FC4FF6FE73C0F264
:100B6C001F03023BB9D0FCE770B5FFF783FF1020E1
:100B7C000121FFF7E1FE40F21C0408200121FFF7E0
:100B8C00DBFEC2F2000441F20000012610252146D2
:100B9C004FF03002C4F201002280A670E570FFF71E
:100BAC00D9FA40F600404FF4C073C4F2010021465C
:100BBC00A670E5702380BDE87040FFF7CBBA00BF8C
:100BCC00002103E00A4B5B584350043109480A4B9F
:100BDC0042189A42F6D3094A02E0002342F8043B39
:100BEC00074B9A42F9D3FFF7BFFFFFF775FF70472A
:100BFC00340C000800000020140000201400002019
:100C0C0020000020FEE70000F8B500BFF8BC08BCCF
:100C1C009E467047F8B500BFF8BC08BC9E467047AE
:040C2C00210100089A
:040C30000D010008AA
:100C3400000000000102030401020304060708097E
:040C44000204060898
:0400000508000BCD17
:00000001FF
